:0400000024EF08F0F1
:1000080000C016F001C015F0E1CF17F0E2CF18F0EC
:100018009DAA74D09EAA72D0AECF9BF1ABA40ED08D
:10002800AB9E010E1D24006E000E1E20016E00C046
:100038001DF001C01EF0AB8E01019B6BABA20FD06F
:10004800AB98AB88010E00016325006E000E642199
:10005800016E00C063F001C064F001019B6B0101F7
:10006800000E9A1902E1010E991916E1C80E000155
:10007800C625E16E000EC721E26EE66A010E736FB7
:10008800000E746FC6C071F0C7C072F0C66BC76B44
:10009800AECF9BF19D9A17D00001C80EC625E16E20
:1000A800000EC721E26E9BC1E6FF010EC625006E59
:1000B800000EC721016E00C0C6F001C0C7F0C6C05F
:1000C80071F0C7C072F0800E006E800EC719005C18
:1000D80002E1C651800812E2020E736F000E746FBF
:1000E8009D9A020EC65D006E000EC759016EC80EBD
:1000F8000024E16E000E0120E26EE66A9DA01FD08A
:100108009EA01DD0010E01019C5D006E000E9D5940
:10011800016E00C09CF101C09DF1000E9D5D02E1E1
:10012800010E9C5D07E29C6B9D6B010E996F000EA2
:100138009A6F9D903C0ECF6EB00ECE6E9E9016C0FC
:1001480000F015C001F017C0E1FF18C0E2FF110070
:0E015800ACB202D00000FCD7B5C1ADFF120062
:0C01660072B201D0FDD7B5C173FF1200CA
:10017200C7B409D01F0EC514016E0150000A03E175
:0A018200010E006E01D0006A1200A9
:10018C00F250026EF29E0500FF6A0150FE6E0050A6
:08019C00FD6E02BEF28E12009E
:1001A40054C0B1F155C0B2F156C0B3F157C0B4F167
:1001B4000101AF6BB06BB051120802E1AF518E0870
:1001C40008E3D5DF005201E004D00101AF4BB02BAE
:1001D400F2D70101120EB05D02E18F0EAF5D03E3B1
:1001E4007B0E006E24D0C580C5A020D0545055107D
:1001F400561057101AE0B151B211B311B4110EE1F7
:100204009FC0E1FFA0C0E2FF050EE66E9DC000F0B6
:100214009EC001F0B9DF010E006E09D0010E01018C
:10022400B15F000EB25BB35BB45BDED7006A120051
:100234009E96AFC1C9FF54C0B0F155C0B1F156C0CC
:10024400B2F157C0B3F1C7A421D054505510561081
:1002540057101BE00101B051B111B211B3110EE1FD
:100264009FC0E1FFA0C0E2FF040EE66E9DC000F057
:100274009EC001F089DF010E006E3AD0010E01012B
:10028400B05F000EB15BB25BB35BDDD754C0B0F1BD
:1002940055C0B1F156C0B2F157C0B3F19EB621D0EA
:1002A40054505510561057101BE00101B051B111B4
:1002B400B211B3110EE19FC0E1FFA0C0E2FF040E32
:1002C400E66E9DC000F09EC001F05EDF010E006E80
:1002D4000FD0010E0101B05F000EB15BB25BB35BE6
:1002E400DDD7C5BC02D0006A03D0C584020E006EFF
:0202F4001200F6
:0402F600C5841200A9
:1002FA0054DF98C1AFF199DF00C0AEF10050FF0A98
:10030A00D8B4C69EADC1AFF190DF00C0AEF1EEDF4A
:06031A00AEC100F012006C
:10032000F00E0101AA15006E0086008000C0ABF13E
:1003300098C1ACF1040E0010AD6FDFDF0D0E0D6E35
:100340000D2EFED798C1ACF1FB0E0101AB15AD6FC0
:10035000D4DF0D0E0D6E0D2EFED7AAC100F00036B3
:100360000090003600900036009000360090F00EAD
:1003700000160086008000C0ABF198C1ACF1040EFD
:1003800000100101AD6FB9DF0D0E0D6E0D2EFED701
:1003900098C1ACF1FB0E0101AB15AD6FAEDF210EC4
:0803A0000D6E0D2EFED71200B8
:1003A8000101AA1D206E080E216E8994F0EC01F05F
:1003B8002032D8B0E3EF01F08984E4EF01F08994AA
:1003C800F0EC01F0212EDCEF01F08984F0EC01F073
:1003D800F0EC01F0FDEF01F01C0E226E00000000B1
:1003E80000000000222EF2EF01F0000000000000E3
:0603F800120000001200DB
:1003FE00086A080E0C6E003408360450085ED8B039
:0E040E0002D00826D89000360C2EF5D712002A
:10041C000101A76BA86BA5C103F0A6C104F0A5C18F
:10042C0005F0A6C106F003C0E9FF04C0EAFFEE50D8
:10043C00200A04E1A751A81101E110D0010EA76F09
:10044C00000EA86F03C0E9FF04C0EAFF05C0E1FF7E
:10045C0006C0E2FFEECFE6FF054A062A03C001F014
:10046C0004C002F0034A042A01C0E9FF02C0EAFFFB
:10047C00EE50000AD8E1A5C100F0A6C101F01200AF
:10048C00A5C102F0A6C103F002C000F003C001F048
:10049C00024A032A00C0E9FF01C0EAFFEE5201E064
:1004AC00F3D70101A551025C006EA6510358016EF1
:0A04BC00010E005E000E015A12004E
:1004C600086A096A100E0C6E0134083609360450A3
:1004D600085E0550D8A0053C095ED8B007D0045088
:1004E60008260550D8B0053C0926D89000360136B6
:0604F6000C2EEAD71200F3
:1004FC00A5C1F6FFA6C1F7FFA7C1F8FF0900F5CF0C
:10050C0000F0005210E0A5C1F6FFA6C1F7FFA7C18D
:10051C00F8FF0900F5CFAAF141DF010EA527000E67
:08052C00A623A723E5D7120066
:100534000B6A0A6A096A00500402F4CF09F0F3CF87
:1005440008F001500502F4CF0BF0F3CF0AF000508D
:100554000502F3500926F4500A22E86A0B220150DE
:100564000402F3500926F4500A22E86A0B2208C058
:1005740000F009C001F00AC002F00BC003F0120041
:0A058400000000000000000012005B
:10058E00A5C1F6FFA6C1F7FFA7C1F8FF0900F5CF79
:10059E0000F0005211E0A5C1F6FFA6C1F7FFA7C1FA
:1005AE00F8FF0900F5CFAAF1B4DE010E0101A5276F
:0A05BE00000EA623A723E4D71200C5
:1005C800030E0C6E950E0D6E0D2EFED70C2EFCD75D
:0205D80012000F
:0E05DA00670E0D6E0D2EFED700000000120001
:1005E800F00E0101A515006E008600C0A7F198C1A4
:1005F800ACF1040E0010AD6F7CDE420E0D6E0D2EB8
:10060800FED7000098C1ACF1FB0E0101A715AD6F34
:1006180070DE420E0D6E0D2EFED700000101A651B0
:10062800010A29E1A5C100F00036009000360090CB
:100638000036009000360090F00E0016008600C0CC
:10064800A7F198C1ACF1040E0010AD6F52DE0D0E8B
:100658000D6E0D2EFED798C1ACF1FB0E0101A7154A
:10066800AD6F47DE1A0E0C6EF80E0D6E0D2EFED70E
:080678000C2EFCD7000012005B
:10068000A9C100F00101A907005228E0A5C1E9FFB6
:10069000A6C1EAFFEE50000A0CE0A5C1E9FFA6C121
:1006A000EAFFA7C1D9FFA8C1DAFFEE50DE1801E1C9
:1006B0000FD0A5C1E9FFA6C1EAFFA7C1D9FFA8C114
:1006C000DAFFDE50EE5C006E016A000E015A08D0BF
:1006D0000101A54BA62BA74BA82BD2D7006A016A14
:0206E000120006
:1006E200A5C1E9FFA6C1EAFFEE500101A71905E184
:1006F200A5C100F0A6C101F010D0A5C100F0A6C1AD
:1007020001F0A54BA62B00C0E9FF01C0EAFFEECF26
:0C07120000F00052E5E1006A016A1200EC
:0C071E00420E0D6E0D2EFED700001200E2
:10072A00A0C101F0010E006E015004E000360090F5
:10073A00FF0FFBD700C0A4F1001E00C0A3F19EC1A9
:10074A00E9FF9FC1EAFF0050EF16120EE9260101E8
:10075A00A26BA251070815E3A2C100F0A1C101F0E2
:10076A00005004E00132019EFF0FFBD7A351EF16A0
:10077A0001A002D0A451EF122BDFA451EF12A22B39
:0C078A00E8D7120EE95EC6DFC5DF1200E2
:100796000101A06BA16B9EC1E9FF9FC1EAFFEE506C
:1007A600000A16E0800EA119006E800E005C02E1C0
:1007B600100EA05D0DE29EC1E9FF9FC1EAFFEECFDC
:1007C600AAF1ABDD01019E4B9F2BA04BA12BE3D7DA
:0207D60012000F
:1007D8000101A26B050EA25D0AE2A251A025E16EFD
:1007E800000EA121E26E200EE66EA22BF3D7A251D5
:1007F800A025E16E000EA121E26EE66AA207A251D1
:10080800A025A36F000EA121A46F0A0E046E000E8E
:10081800056E9EC100F09FC101F051DE08C000F0D6
:1008280009C001F0300E0026A3C1E1FFA4C1E2FF18
:1008380000C0E6FF0A0E046E000E056E9EC100F0B1
:100848009FC101F03CDE00C09EF101C09FF1000E87
:10085800011802E1000E001801E102D0A207CFD76B
:0208680012007C
:10086A000D0E0101B56F73DC0A0E0101B56F6FDC65
:02087A0012006A
:10087C000101A16B9FAF09D0010EA16F2D0E486F26
:10088C009E1F9F1F9E4B9F2B03D0A16B200E486F6A
:10089C009EC100F09FC101F001320032019E013275
:1008AC000032019E01320032019E01320032019E63
:1008BC0000C0A0F10A0E046E9CDD0A0E046E99DDD8
:1008CC0008C000F0300E0024016E01C049F1015047
:1008DC00300A02E1200E496F0A0E046EA0C100F02E
:1008EC0088DD08C000F0300E00244A6F0F0E9E15F4
:1008FC00006E9FC101F0000E0116710E046E020E07
:10090C00056E12DE00C0A2F101C0A3F12E0E4B6FDA
:10091C00E80E046E030E056EA2C100F0A3C101F037
:10092C00CCDD300E00244C6F640E046E000E056E90
:10093C00A2C100F0A3C101F0C0DD0A0E046E000ECE
:10094C00056EBBDD08C000F009C001F0300E0024BC
:10095C004D6F4E6B4F6B506B490EA56F010EA66F12
:08096C0057DDA1C100F01200EB
:100974009EC1E9FF9FC1EAFFEE5000080AE29EC152
:10098400E9FF9FC1EAFFEECFAAF10CDD9E4B9F2B3E
:04099400EFD7120087
:10099800300ECD6E9E903C0ECF6EB00ECE6E9EC1C8
:1009A8009CF19FC19DF10101996B9A6B9E909D905E
:0609B800CD809D801200BD
:1009BE00016A026A800E0218006E800E000A005C48
:1009CE0002E17F0E015C0AE2C80E0124E16E000E08
:1009DE000220E26EE66A014A022AECD7AECF9BF104
:1009EE000001C86B01019B6B0001C66BC76B716B7D
:0A09FE00726B736B746B9D8A12001C
:100A0800A0C101F0010E006E015004E00036009014
:100A1800FF0FFBD700C0A2F1001E9EC1E9FF9FC1D6
:100A2800EAFF0050EF16120EE9260050EF16C8DD57
:100A38000101A251EF12120EE95ECBDDA251EF14B3
:100A4800A16FA151000A000ED8A4010EA16FB8DD54
:060A5800A1C100F0120034
:100A5E00A0C1F6FFA1C1F7FFA2C1F8FF0900F5CFB3
:100A6E0000F0005218E0A0C1F6FFA1C1F7FFA2C12D
:100A7E00F8FF0900F5CF00F09EC1E1FF9FC1E2FF34
:100A8E0000C0E6FF01019E4B9F2B010EA027000E1A
:100A9E00A123A223DDD79EC1E1FF9FC1E2FFE66A3B
:020AAE00120034
:100AB0009EC1F6FF9FC1F7FFA0C1F8FF0900F5CF67
:100AC00000F0005212E09EC1F6FF9FC1F7FFA0C1E7
:100AD000F8FF0900F5CFB5F1ACEC00F0010E010113
:0C0AE0009E27000E9F23A023E3D71200E6
:100AEC00000E01019F1902E1000E9E1934E09EC117
:100AFC00E9FF9FC1EAFFEE522EE0A0C1A5F1A1C112
:100B0C00A6F1BEDC00C0A9F19EC1A5F19FC1A6F162
:100B1C00A0C1A7F1A1C1A8F1ADDD000E011802E141
:100B2C00000E001805E19EC100F09FC101F015D028
:100B3C00010E01019E25A56F000E9F21A66FA0C17D
:100B4C00E9FFA1C1EAFFEECFA7F1C5DD00C09EF120
:0C0B5C0001C09FF1C5D7006A016A1200B9
:100B6800580E0001996F010E9A6FB50E9B6F010E1A
:100B78009C6FFF0E916FFF0E926F000E936F000E29
:100B8800946FFF0E896FFF0E8A6F000E8B6F000E39
:100B98008C6FFF0E8D6FFF0E8E6F000E8F6F000E25
:100BA800906FAC8A900EAB6E948E949C9EAA03D0E4
:080BB800AECF00F0FBD71200E4
:100BC0002AD0800E0101A56F010EA66F0DDD630E08
:100BD0000101A56F1F0EA66F000EA76FD8DC800E57
:100BE0000101A56F010EA66FFFDC22D0C00E01012E
:100BF000A56F010EA66FF8DC300E0101A56F1F0E68
:100C0000A66F000EA76FC3DCC00E0101A56F010E19
:100C1000A66FEADC0DD0000E01019F1902E1010E62
:100C20009E19CFE0000E9F1902E1020E9E19DEE030
:020C30001200B0
:100C32000D0E0101AA6FD4EC01F00A0EAA6FD4ECDA
:040C420001F01200AB
:100C46000900F5CFE6FF0006FBE10106F9E1120017
:100C5600806A0F01386B3881230E926E92988988CC
:100C66009296898692948984396BFF0E816E8F0ED7
:100C7600936EF19E3A6B826AFF0E946E949C9492E8
:080C860094908B80606A12005B
:100C8E0000016F6B706B800E7019006E800E005C31
:100C9E0002E10A0E6F5D27E2030E006E000E016E7A
:100CAE006FC004F070C005F03EDC240E0024E96E27
:100CBE00000E0120EA6EEECFA5F1EECFA6F1EECF3B
:100CCE00A7F115DC070E0B6E170E0C6E6A0E0D6E6D
:100CDE000D2EFED70C2EFCD70B2EFAD700000001DE
:080CEE006F4B702BD0D71200F0
:100CF6009EC100F00032009E0032009E0032009E2F
:100D06000032009EB50E0024F66E1F0EF76E000E22
:100D1600F722000EF86E000EF8220900F5CF00F05B
:100D26009FC1E1FFA0C1E2FF00C0E6FF010E010185
:100D36009F25E16E000EA021E26E0F0E9E15006E3D
:100D4600B50E0024F66E1F0EF76E000EF722000E8B
:100D5600F86E000EF8220900F5CF00F000C0E6FF9D
:100D6600020E9F25E16E000EA021E26EE66A1200D9
:100D7600A0C101F0010E006E015004E000360090A3
:100D8600FF0FFBD700C0A4F1001C0101A36FA26BEB
:100D96009EC1E9FF9FC1EAFFA16BA151070822E3AB
:100DA600A351EF16120EE926A351EF16C2EC02F07C
:100DB600A451EF12C2EC02F0120EE95EA451EF1438
:100DC600006E0CE0A1C101F0010E006E015004E0BE
:100DD60000360090FF0FFBD70050A2139DDC9CDC71
:0A0DE600A12BDBD7A2C100F0120020
:100DF0000101A16B9EC1E9FF9FC1EAFFEECFA0F107
:100E0000A051000A0FE0A0C1B5F1ACEC00F0010167
:100E1000A12BA1519E25E96E000E9F21EA6EEECF17
:060E2000A0F1EED7120064
:100E2600720E0001816F010E826F000E836F000E3D
:100E3600846FA40E856F010E866F000E876F000EFD
:100E4600886FFF0E7D6FFF0E7E6F000E7F6F000EA8
:100E5600806FFF0E756FFF0E766FFF0E776FFF0EBA
:100E6600786F340E796F020E7A6FAF0E7B6F010EBC
:100E76007C6FF60E956F020E966F000E976F000E42
:100E8600986F949894968B988B9694889486C79E20
:080E9600C79C380EC66E120065
:100E9E00200E0101AA6FD4EC01F0200EAA6FD4EC43
:100EAE0001F0300EAA6FD4EC01F0030E0B6E080E9B
:100EBE000C6E770E0D6E0D2EFED70C2EFCD70B2E54
:100ECE00FAD7300EA56FA66BF4EC02F0310E0101CD
:100EDE00AA6FD4EC01F0820E0C6EDD0E0D6E0D2E8F
:100EEE00FED70C2EFCD700000000300EA56FA66BAF
:100EFE00F4EC02F0320E0101AA6FD4EC01F0820E76
:100F0E000C6EDD0E0D6E0D2EFED70C2EFCD70000D6
:100F1E000000300EA56FA66BF4EC02F0330E01014B
:100F2E00AA6FD4EC01F0820E0C6EDD0E0D6E0D2E3E
:100F3E00FED70C2EFCD700000000250EA56FA66B69
:100F4E00F4EC02F0340E0101AA6FD4EC01F0680E3D
:100F5E000C6EE40E0D6E0D2EFED70C2EFCD700007F
:100F6E00280EA56F010EA66FF4EC02F0350E0101EE
:100F7E00AA6FD4EC01F00B0E0C6E620E0D6E0D2EE0
:100F8E00FED70C2EFCD70000080EA56F010EA66F23
:100F9E00F4EC02F0360E0101AA6FD4EC01F00B0E48
:100FAE000C6E620E0D6E0D2EFED70C2EFCD70000B1
:100FBE00010EA56F010EA66FF4EC02F0370E0101C3
:100FCE00AA6FD4EC01F0680E0C6EE40E0D6E0D2EB1
:100FDE00FED70C2EFCD70000060EA56F010EA66FD5
:100FEE00F4EC02F0380E0101AA6FD4EC01F00B0EF6
:100FFE000C6E620E0D6E0D2EFED70C2EFCD7000061
:10100E000C0EA56F010EA66FF4EC02F0390E010165
:10101E00AA6FD4EC01F00D0EAA6FD4EC01F00A0EFB
:10102E00AA6FD4EC01F00B0E0C6E620E0D6E0D2E2F
:0A103E00FED70C2EFCD700001200B4
:1010480027EC10F09B6A720ED36E9B9CD26AD3B4C5
:1010580001D0FDD7FCDD206A216A226A236AE5DD1A
:1010680000016F6B706B800E7019006E800E005C53
:1010780002E1040E6F5D21E289968988070E0B6EE6
:10108800170E0C6E6A0E0D6E0D2EFED70C2EFCD7A9
:101098000B2EFAD7000089868998070E0B6E170E5B
:1010A8000C6E6A0E0D6E0D2EFED70C2EFCD70B2E75
:1010B800FAD700006F4B702BD6D789868998656B55
:1010C800666B636B646B1D6A1E6A616B626BAB6AED
:1010D800AB88AB8EAB8A6B6B6C6B708201019B6BC0
:1010E8008998480E00016D6F010E6E6FB886010E6B
:1010F800B06EA00EAF6EAC8433DD050E0B6E0F0E16
:101108000C6EF10E0D6E0D2EFED70C2EFCD70B2E8D
:10111800FAD7B9DD899489DD090EA56F1F0EA66F70
:10112800000EA76F7EEC02F00A0EC86E78DE0B0E7A
:101138000B6E260E0C6E5D0E0D6E0D2EFED70C2E50
:10114800FCD70B2EFAD7000000004A0E0101986F59
:10115800AC0EA56F1E0EA66F000EA76F7EEC02F0F8
:1011680064DD4A0E1F6E920EA56F1E0EA66F000E4E
:10117800A76F7EEC02F08FDE58DD010EAA6F90ECAF
:1011880001F0010E01019E6F000E9F6F15DD520EDA
:101198000101A56F1F0EA66F000EA76FC7EC02F026
:1011A800290E0B6E960E0C6E7F0E0D6E0D2EFED751
:1011B8000C2EFCD70B2EFAD7020E0101A56F1E0EBE
:1011C800A66F000EA76F7EEC02F06DC09EF16EC098
:1011D8009FF1410E0101A06F1F0EA16F000EA26FBB
:1011E8003ADC6DC09EF16EC09FF1BAEC04F01DDDD3
:1011F800020E9E6F000E9F6FDFDC6DC09EF16EC009
:101208009FF1CBEC03F0290E0B6E960E0C6E7F0E41
:101218000D6E0D2EFED70C2EFCD70B2EFAD7020E14
:101228009E6F000E9F6FC8DC010E01019E6F000EBD
:101238009F6FC2DC740E0101A56F1F0EA66F000E12
:10124800A76FC7EC02F0290E0B6E960E0C6E7F0E80
:101258000D6E0D2EFED70C2EFCD70B2EFAD79D80C7
:101268009D8AF28CF28EBE0E0101A56F1D0EA66F2F
:10127800000EA76F7EEC02F08B900B0E0B6E260E05
:101288000C6E5D0E0D6E0D2EFED70C2EFCD70B2EA0
:10129800FAD700000000450E01019E6F200E9F6FD7
:1012A800000EA06F01DC030E0B6E080E0C6E770E9D
:1012B8000D6E0D2EFED70C2EFCD70B2EFAD7EE0E88
:1012C80001019E6F1F0E9F6F000EA06F58EC05F076
:1012D800030E0B6E080E0C6E770E0D6E0D2EFED7DC
:1012E8000C2EFCD70B2EFAD7F90E01019E6F1F0E9C
:1012F8009F6F000EA06F58EC05F0030E0B6E080EE2
:101308000C6E770E0D6E0D2EFED70C2EFCD70B2E05
:10131800FAD7170E01019E6F200E9F6F000EA06F67
:1013280058EC05F0030E0B6E080E0C6E770E0D6E62
:101338000D2EFED70C2EFCD70B2EFAD7DC0E010192
:10134800A56F1C0EA66F000EA76F7EEC02F0200E94
:101358000101A56F200EA66F000EA76F7EEC02F0AC
:10136800DFEC04F0140E01019E6F000E9F6FCCECB1
:1013780004F0280E9E6F200E9F6F000EA06F58EC91
:1013880005F0050E0B6E0F0E0C6EF10E0D6E0D2E88
:10139800FED70C2EFCD70B2EFAD7000E01019A1996
:1013A80002E1000E991908E1000E0001741902E12A
:1013B800000E731901E1F1D70101996B9A6B000EC8
:1013C8000001741902E1010E73190AE0800E006E23
:1013D800800E7219005C02E17151020801E30DD020
:1013E8000101996B9A6B21DCC80E9E6F000E9F6FEE
:1013F800BAEC04F01ADCAECF9BF18B800B0E0B6EAF
:10140800260E0C6E5D0E0D6E01010D2EFDD70C2EF5
:10141800FBD70B2EF9D700000000780EA56F1E0E23
:10142800A66F000EA76F7EEC02F0030E0B6E080E7F
:101438000C6E770E0D6E0D2EFED70C2EFCD70B2ED4
:10144800FAD70001676B686B800E01019E6F0F0E63
:101458009F6F010EA06F04EC05F0020E0C6E4B0E90
:101468000D6E0D2EFED70C2EFCD7800E9E6F0F0E24
:101478009F6F010EA06F330EA16F95EC03F0020E63
:101488000C6E4B0E0D6E0D2EFED70C2EFCD7800E5B
:101498009E6F0F0E9F6F010EA06F69DC00C09BF15D
:1014A800020E0C6E4B0E0D6E0D2EFED70C2EFCD7B9
:1014B800C50EA56F1F0EA66F000EA76F7EEC02F07B
:1014C800480E00016D6F010E6E6F6DC0E1FF6EC0BA
:1014D800E2FFE66A9BC19EF16DC09FF16EC0A0F16C
:1014E80006DC6DC09EF16EC09FF1BAEC04F0380EB8
:1014F8000101A56F200EA66F000EA76F7EEC02F00B
:1015080000016F6B706B800E7019006E800E005CAE
:1015180002E1060E6F5D29E2800E01019E6F0F0E3B
:101528009F6F010EA06F23DC00C09BF1020E0C6EB2
:101538004B0E0D6E0D2EFED70C2EFCD76DC0E1FFA5
:101548006EC0E2FFE66A9BC19EF16DC09FF16EC05E
:10155800A0F17BEC06F06DC09EF16EC09FF1BAEC75
:1015680004F000016F4B702BCED7300E0101A56F30
:10157800200EA66F000EA76F7EEC02F0800E010110
:101588009E6F0F0E9F6F010EA06FBBEC06F000C0A0
:101598009BF16DC0E1FF6EC0E2FFE66A9BC19EF160
:1015A8006DC09FF16EC0A0F17BEC06F06DC09EF19E
:1015B8006EC09FF1BAEC04F019EC06F00001676BFD
:1015C800686B696B6A6B196A899889888B80030EC6
:1015D8000B6E080E0C6E770E0D6E0D2EFED70C2EB0
:1015E800FCD70B2EFAD74A0E01019E6F000E9F6F93
:1015F800030EA06F200EA16F000EA26F2FEC05F056
:1016080019C000F00036009000500A0F016E01C0AA
:10161800A3F0000E015CD8A0DED0640E0001A35D2B
:10162800D8B0D9D00A0E046EA3C000F0FFEC01F0C8
:10163800300E00244F6E0A0E046EA3C000F0FFECBB
:1016480001F008C000F0300E0024506E8B900B0E95
:101658000B6E260E0C6E5D0E0D6E0D2EFED70C2E2B
:10166800FCD70B2EFAD7000000001D0E0101A56F54
:101678001F0EA66F000EA76F7EEC02F04A0E010146
:101688009E6F000E9F6FBAEC04F00A0E01019E6F68
:10169800000E9F6FCCEC04F0DFEC04F04A0E010161
:1016A8009E6F000E9F6FF8EC06F0020E0B6E040E94
:1016B8000C6EBA0E0D6E0D2EFED70C2EFCD70B2E0F
:1016C800FAD700000101000E9A1902E1000E9919DB
:1016D80008E1000E0001741902E1000E731901E11E
:1016E800F1D70101996B9A6B000E0001741902E1A0
:1016F800010E73190AE0800E006E800E7219005CEC
:1017080002E17151070801E33BD00D0E0101A56FFD
:10171800200EA66F000EA76F7EEC02F0C80E010126
:101728009E6F000E9F6FBAEC04F0C80E01019E6F09
:10173800000E9F6F1A0EA06F000EA16F76EC05F0D9
:1017480000C0A1F001C0A2F0000E026E0150025CC0
:1017580002E1005000080AE2D50E0101A56F1F0E34
:10176800A66F000EA76F7EEC02F009D0220E0101D1
:10177800A56F1E0EA66F000EA76F7EEC02F009D0B3
:10178800950E0101A56F1F0EA66F000EA76F7EECC8
:1017980002F08B80040E0B6E0C0E0C6E330E0D6E69
:1017A8000D2EFED70C2EFCD70B2EFAD7000000000A
:1017B800F40E0101A56F1E0EA66F000EA76F7EEC3A
:1017C80002F04FC0AAF1D4EC01F050C0AAF1D4EC59
:1017D80001F019EC06F00101280E9E6F000E9F6FB4
:1017E800CCEC04F0DFEC04F0850E01019E6F1F0EB7
:1017F8009F6F000EA06F58EC05F0030E0B6E080EDD
:101808000C6E770E0D6E0D2EFED70C2EFCD70B2E00
:10181800FAD7000E01019A1902E1000E991908E1A0
:10182800000E0001741902E1000E731901E1F1D7ED
:101838000B0E0B6E260E0C6E5D0E0D6E00010D2E3E
:10184800FDD70C2EFBD70B2EF9D700000000000E99
:10185800741902E1010E73190AE0800E006E800E01
:101868007219005C02E17151040801E3CDD0C80E81
:1018780001019E6F000E9F6F450EA06F000EA16FB5
:1018880076EC05F000C0A1F001C0A2F0000E026ED7
:101898000150025C02E10050000817E20001F86BF9
:1018A800E20E0101A56F1F0EA66F000EA76F7EEC5A
:1018B80002F0CD0E01019E6F000E9F6FBAEC04F08E
:1018C80019EC06F00001A16BA26BC80E01019E6F16
:1018D800000E9F6F580EA06F000EA16F76EC05F0FA
:1018E80000C0A1F001C0A2F0000E026E0150025C1F
:1018F80002E10050000817E20001E86B3F0E010109
:10190800A56F200EA66F000EA76F7EEC02F0CC0E1E
:1019180001019E6F000E9F6FBAEC04F019EC06F0FF
:101928000001A16BA26BC80E01019E6F000E9F6F94
:101938005D0EA06F000EA16F76EC05F000C0A1F05F
:1019480001C0A2F0000E026E0150025C02E10050DC
:10195800000857E20001CF6BA1C09EF1A2C09FF121
:10196800BAEC04F0040E0001A125E96E000EA221D4
:10197800EA6EEE503D0A45E1030EA125E96E000E20
:10198800A221EA6EEECFA3F034D0050EA125E96EB0
:10199800000EA221EA6EEE50310AD8B48998050EDD
:1019A800A125E96E000EA221EA6EEE50300AD8B4E5
:1019B800898827D0050EA125E96E000EA221EA6EBE
:1019C800EE50310AD8B48996050EA125E96E000EAD
:1019D800A221EA6EEE50300AD8B4898612D0A50E3C
:1019E8000101A56F1F0EA66F000EA76F7EEC02F017
:1019F80008D00001A351520AC8E0A351560ADAE000
:101A0800EED70001A16BA26B0101486B800E9E6F9F
:101A18000F0E9F6F010EA06F04EC05F0800E9E6FF5
:101A28000F0E9F6F010EA06FCC0EA16F95EC03F007
:101A3800800E9E6F0F0E9F6F010EA06F440EA16F58
:101A480095EC03F0020E0C6E4B0E0D6E0D2EFED7AC
:101A58000C2EFCD7800E9E6F0F0E9F6F010EA06F8D
:101A680004EC05F0800E9E6F0F0E9F6F010EA06FA5
:101A7800CC0EA16F95EC03F0800E9E6F0F0E9F6F3A
:101A8800010EA06FBE0EA16F95EC03F0340E0C6E24
:101A9800F10E0D6E0D2EFED70C2EFCD700000000A7
:101AA800800E9E6F0F0E9F6F010EA06FBBEC06F0AD
:101AB80000C0C4F0000E0001C56F800E01019E6FCA
:101AC8000F0E9F6F010EA06FBBEC06F000C002F076
:101AD800016A01500001C4270250C523430EA46FB8
:101AE800480EA56F4FC0A6F050C0A7F0200EA86FF3
:101AF80067C09EF168C09FF1A80E0101A06F000E9B
:101B0800A16FECEC03F0200E0001AE6FAF6BC4C008
:101B18009EF1C5C09FF13EEC04F000C0A3F0A40EF6
:101B28009E6F000E9F6FF8EC06F0480E9E6F010E38
:101B38009F6FF8EC06F035EC04F0A40E01019E6FDF
:101B4800000E9F6FBAEC04F0480E01019E6F010E63
:101B58009F6FBAEC04F019EC06F09D90192A195001
:101B68000308D8A0196A000E0001741902E1020ED8
:101B780073190CE15D0E0101A56F1E0EA66F000E14
:101B8800A76F7EEC02F00001736B746B674B682BD8
:041B98002AD5FFD774
:10204E0010EE24F0210E006E010E016EE10EF66E02
:10205E001D0EF76E000EF86E23EC06F010EE19F062
:10206E00040E006E010E016E4A0EF66E200EF76E15
:10207E00000EF86E23EC06F010EE45F01C0E006E0E
:10208E00010E016E410EF66E1E0EF76E000EF86E0C
:06209E0023EC06F0120025
:101B9C00204469726563746F72793A20433A5C5FD2
:101BAC004D696B726F435C5F4D657350726F6A6504
:101BBC0074735F4D696B726F435C5F484331325F86
:101BCC005472616E736365697665725F3433334D3D
:051BDC00687A0D0A000B
:101BE1002050726F6A6574203A205031384632367F
:101BF1004B32325F436F6E63656E747261746575EB
:101C0100725F34785F484331325F4655335F39360E
:101C110030305F3139313130392E6D637070690D7B
:021C21000A00B7
:101C230020536F75726365205031384632364B321C
:101C3300325F436F6E63656E747261746575725F54
:101C430034785F484331325F56325F365F465533EF
:101C53005F393630305F3139313130392E630D0A17
:011C63000080
:101C640020464F534320696E7465726E652020319F
:101C7400364D487A20766961205031384632364BE9
:101C840032325F464F53435F696E7465726E655FAF
:0F1C940031364D687A2E6366677363680D0A00F8
:101CA30020506F7274204861726420554152543140
:101CB30020393630302C4E2C382C3120706F757211
:101CC300204843313220285243363D545820524352
:091CD300373D525829200D0A008A
:101CDC000D0A204C656374757265205365747469C4
:101CEC006E6720204843313220636F6E63656E74DB
:101CFC007261746575722073757220426173652010
:071D0C005049430D0A2000BD
:101D1300205465726D696E616C207375722054581E
:101D230020554152543320313932303062647320AC
:101D330041534D20524132206F75747075740D0AF2
:011D4300009F
:101D440020436F6E666967203A2050313846323638
:101D54004B32325F464F53435F696E7465726E65F2
:101D64005F31364D687A2E6366677363680D0A00C7
:101D7400204D435520203A31384632364B323220FA
:101D8400416C696D2E203D2020332E3620E0203416
:061D94002E38560D0A0076
:101D9A00205241303D41444320205241313D4F576A
:101DAA00532073656E736F72204453313842323058
:041DBA00200D0A00EE
:101DBE0020496E69742053657474696E67202043E0
:101DCE00616E616C203130206D6F64652020465548
:031DDE00332000AF
:101DE1009C1B00E11B00741D00441D00641C00A32A
:101DF1001C009A1D00231C00131D00DD1E00C51EC2
:011E010000E0
:101E02002045637269742E207375722032656D20CD
:101E12006C69676E65206475204C4344203A20004B
:101E220020504220737572204368616E67656D654C
:0F1E32006E742064652043616E616C200D0A00A0
:051E41004D73673D0038
:0A1E460041542B433031300D0A00E7
:041E5000000000008E
:051E54004B4D4C2C0079
:041E59004C454400B0
:101E5D00205042206465626F7264656D656E7420FA
:0B1E6D0062756666657231200D0A0088
:101E78002054657374207265676973747265732082
:0A1E8800445331384232300D0A0095
:101E920020496E697420446973706C6179204C43E7
:0A1EA200442032783136203A200047
:101EAC00204954205541525431205243362026208B
:091EBC0054696D6572310A0D00D4
:101EC500204C616E67616765204D696B726F4320B9
:081ED500372E3530200D0A0004
:101EDD0020454550524F4D206E6F6E207574696CC4
:071EED006973E9650D0A00AD
:101EF400E0206C2765636F75746520647520434129
:051F04004E414C2000DD
:101F090020496E69742049324331203430304B689E
:041F19007A0D0A0033
:101F1D000D0A20536574206368616E6E656C203AFE
:031F2D0020200071
:101F300020202020202020202020202020202020A1
:011F400000A0
:101F41007061756C666A756A6F2030313233343571
:011F5100008F
:101F520048656C6C6F204920616D20616C69766503
:011F6200007E
:101F6300202020202020202020202020202020206E
:011F7300006D
:101F74007061756C666A756A6F2E667265652E6629
:011F8400005C
:101F850057616974696E67206D736720210D0A00BA
:101F9500204E4F20726573706F6E7365200D0A00B9
:101FA5004E6F20636F6D7072656E646F200D0A0051
:101FB500303132333435363738394142434445467A
:101FC5002046616D696C7920436F6465203A200075
:0D1FD5002043616E616C204F4B200D0A000F
:0C1FE2004D7367207265E775203A2000FF
:0B1FEE0041542B42393630300D0A0000
:0A1FF90041542B433031300D0A0033
:0A20030041542B433030300D0A0029
:0A200D00205265746F75723A2000CE
:0920170041542B4655330D0A001B
:0820200041542B52580D0A0037
:0820280041542B52580D0A002F
:0820300020204352433D200033
:07203800204944313D200066
:06203F004750533D200054
:0520450041540D0A00EA
:01204A000095
:03204B004F4B00F8
:020000040030CA
:0D000100231F3CFFBF81FF0FC00FE00F4029
:00000001FF
